:04000003F000B3D185
:020000040000FA
:1000000000040020810A000015070000610A0000BA
:100010001F07000029070000330700000000000050
:10002000000000000000000000000000A50A000021
:100030003D070000000000004707000051070000D6
:100040005B070000650700006F07000079070000EC
:10005000830700008D07000097070000A10700003C
:10006000AB070000B5070000BF070000C90700008C
:10007000D3070000DD070000E7070000F1070000DC
:10008000FB070000050800000F0800001908000029
:10009000230800002D080000370800004108000078
:1000A0004B080000550800005F08000069080000C8
:1000B000730800007D080000870800009108000018
:1000C0009B080000A5080000AF080000B908000068
:1000D000C3080000CD080000D7080000E1080000B8
:1000E000EB080000F5080000FF0800000909000007
:1000F000130900001D090000270900003109000054
:100100003B0900001FB500F003F88DE80F001FBD8C
:1001100000F0ACBC40F6FC7108684FF01022401CA7
:1001200008D00868401C09D00868401C04D0086842
:1001300000F037BA9069F5E79069F9E7704770B554
:100140000B46010B184400F6FF70040B4FF0805073
:100150000022090303692403406943431D1B104621
:1001600000F048FA29462046BDE8704000F042BA47
:10017000F0B54FF6FF734FF4B4751A466E1E11E0DA
:10018000A94201D3344600E00C46091B30F8027B3B
:10019000641E3B441A44F9D19CB204EB134394B25D
:1001A00004EB12420029EBD198B200EB134002EBB2
:1001B000124140EA0140F0BDF34992B00446D1E952
:1001C0000001CDE91001FF224021684600F0F4FB58
:1001D00094E80F008DE80F00684610A902E004C8FB
:1001E00041F8042D8842FAD110216846FFF7C0FF7C
:1001F0001090AA208DF8440000F099F9FFF78AFFCB
:1002000040F6FC7420684FF01025401C0FD0206889
:1002100010226946803000F078F92068401C08D030
:100220002068082210A900F070F900F061F9A869AF
:10023000EEE7A869F5E74FF080500369406940F6A2
:10024000FC71434308684FF01022401C06D0086838
:1002500000F58050834203D2092070479069F7E788
:100260000868401C04D00868401C03D00020704778
:100270009069F9E70420704770B504460068C34DE3
:10028000072876D2DFE800F033041929631E250021
:10029000D4E9026564682946304600F062F92A46CE
:1002A0002146304600F031F9AA002146304600F0E0
:1002B00057FB002800D0032070BD00F009FC4FF46C
:1002C000805007E0201D00F040F90028F4D100F034
:1002D000FFFB60682860002070BD241D94E80700C3
:1002E000920000F03DFB0028F6D00E2070BDFFF715
:1002F000A2FF0028FAD1D4E901034FF0805100EBAE
:10030000830208694D69684382420ED840F6F8704E
:1003100005684FF010226D1C09D0056805EB8305B8
:100320000B6949694B439D4203D9092070BD55694A
:10033000F4E70168491C03D00068401C02D003E0C8
:100340005069FAE70F2070BD2046FFF735FFFFF731
:1003500072FF0028F7D1201D00F0F7F80028F2D135
:1003600060680028F0D100F0E2F8FFF7D3FE00F05B
:10037000BFF8072070BD10B50C46182802D0012028
:10038000086010BD2068FFF777FF206010BD41684E
:10039000054609B1012700E0002740F6F8742068FF
:1003A0004FF01026401C2BD02068AA68920000F065
:1003B000D7FA38B3A86881002068401C27D020688D
:1003C000FFF7BDFED7B12068401C22D026684FF051
:1003D0008050AC686D68016942695143A9420DD9EA
:1003E000016940694143A14208D92146304600F0E5
:1003F000B8F822462946304600F087F800F078F831
:100400007069D2E700F093F8FFF784FEF6E77069B1
:10041000D6E77669DBE740F6FC7420684FF01026DB
:10042000401C23D02068401C0CD02068401C1FD0EA
:100430002568206805F18005401C1BD027683879A5
:10044000AA2819D040F6F8700168491C42D001680A
:10045000491C45D00168491C3ED001680968491C07
:100460003ED00168491C39D000683EE0B069DAE747
:10047000B569DEE7B769E2E710212846FFF778FEA5
:100480003968814222D12068401C05D0D4F8001080
:1004900001F18002C03107E0B169F9E730B108CA63
:1004A00051F8040D984201D1012000E000208A4259
:1004B000F4D158B1286810B1042803D0FEE72846CB
:1004C000FFF765FF3149686808600EE0FFF722FE1C
:1004D00000F00EF87169BBE77169BFE7706904E06D
:1004E0004FF480500168491C01D000F0CBFAFEE7C0
:1004F000BFF34F8F26480168264A01F4E06111439B
:100500000160BFF34F8F00BFFDE72DE9F0411746B3
:100510000D460646002406E03046296800F054F8EF
:10052000641C2D1D361DBC42F6D3BDE8F08140F69B
:10053000FC700168491C04D0D0F800004FF48051D1
:10054000FDE54FF010208069F8E74FF080510A690F
:10055000496900684A43824201D810207047002050
:10056000704770B50C4605464FF4806608E0284693
:1005700000F017F8B44205D3A4F5806405F5805562
:10058000002CF4D170BD0000F40A0000000000202F
:100590000CED00E00400FA05144801680029FCD0C5
:1005A0007047134A0221116010490B68002BFCD0E0
:1005B0000F4B1B1D186008680028FCD0002010603D
:1005C00008680028FCD07047094B10B501221A605A
:1005D000064A1468002CFCD0016010680028FCD08A
:1005E0000020186010680028FCD010BD00E4014015
:1005F00004E5014070B50C46054600F073F810B9EB
:1006000000F07EF828B121462846BDE8704000F091
:1006100007B821462846BDE8704000F037B8000012
:100620007FB5002200920192029203920A0B000B06
:100630006946012302440AE0440900F01F0651F80C
:10064000245003FA06F6354341F82450401C8242F8
:10065000F2D80D490868009A10430860081D016827
:10066000019A1143016000F03DF800280AD00649C4
:1006700010310868029A10430860091D0868039A3F
:10068000104308607FBD00000006004030B50F4CED
:10069000002200BF04EB0213D3F800582DB9D3F8A1
:1006A000045815B9D3F808581DB1521C082AF1D3C3
:1006B00030BD082AFCD204EB0212C2F80008C3F8CD
:1006C00004180220C3F8080830BD000000E0014013
:1006D0004FF08050D0F83001082801D0002070473A
:1006E000012070474FF08050D0F83011062905D016
:1006F000D0F83001401C01D0002070470120704725
:100700004FF08050D0F830010A2801D00020704707
:100710000120704708208F490968095808471020B0
:100720008C4909680958084714208A4909680958FA
:100730000847182087490968095808473020854923
:100740000968095808473820824909680958084744
:100750003C20804909680958084740207D490968BC
:100760000958084744207B49096809580847482028
:1007700078490968095808474C207649096809589A
:10078000084750207349096809580847542071499F
:1007900009680958084758206E49096809580847E8
:1007A0005C206C4909680958084760206949096854
:1007B00009580847642067490968095808476820AC
:1007C00064490968095808476C2062490968095852
:1007D000084770205F4909680958084774205D4937
:1007E00009680958084778205A490968095808478C
:1007F0007C205849096809580847802055490968EC
:10080000095808478420534909680958084788202F
:1008100050490968095808478C204E490968095809
:10082000084790204B4909680958084794204949CE
:10083000096809580847982046490968095808472F
:100840009C204449096809580847A0204149096883
:1008500009580847A4203F49096809580847A820B3
:100860003C49096809580847AC203A4909680958C1
:100870000847B0203749096809580847B420354966
:10088000096809580847B8203249096809580847D3
:10089000BC203049096809580847C0202D4909681B
:1008A00009580847C4202B49096809580847C82037
:1008B0002849096809580847CC2026490968095879
:1008C0000847D0202349096809580847D4202149FE
:1008D000096809580847D8201E4909680958084777
:1008E000DC201C49096809580847E02019490968B3
:1008F00009580847E4201749096809580847E820BB
:100900001449096809580847EC2012490968095830
:100910000847F0200F49096809580847F4200D4995
:10092000096809580847F8200A490968095808471A
:10093000FC2008490968095808475FF48070054998
:10094000096809580847000003480449024A034B54
:100950007047000000000020000B0000000B0000AA
:1009600040EA010310B59B070FD1042A0DD310C82C
:1009700008C9121F9C42F8D020BA19BA884201D97E
:10098000012010BD4FF0FF3010BD1AB1D30703D0C6
:10099000521C07E0002010BD10F8013B11F8014B7C
:1009A0001B1B07D110F8013B11F8014B1B1B01D198
:1009B000921EF1D1184610BD02F0FF0343EA032254
:1009C00042EA024200F005B87047704770474FF0A6
:1009D00000020429C0F0128010F0030C00F01B800C
:1009E000CCF1040CBCF1020F18BF00F8012BA8BF1A
:1009F00020F8022BA1EB0C0100F00DB85FEAC17CDE
:100A000024BF00F8012B00F8012B48BF00F8012B90
:100A100070474FF0000200B51346944696462039C1
:100A200022BFA0E80C50A0E80C50B1F12001BFF4A7
:100A3000F7AF090728BFA0E80C5048BF0CC05DF80D
:100A400004EB890028BF40F8042B08BF704748BF5B
:100A500020F8022B11F0804F18BF00F8012B7047CF
:100A6000014B1B68DB6818470000002009480A4951
:100A70007047FFF7FBFFFFF745FB00BD20BFFDE719
:100A8000064B1847064A1060016881F308884068E1
:100A900000470000000B0000000B000017040000DE
:100AA000000000201EF0040F0CBFEFF30881EFF3ED
:100AB0000981886902380078182803D100E0000015
:100AC000074A1047074A12682C3212681047000084
:100AD00000B5054B1B68054A9B58984700BD0000B0
:100AE0007703000000000020F00A0000040000006E
:100AF000001000000000000000FFFFFF0090D00386
:1010000080130020B157020069C00000175702008A
:1010100069C0000069C0000069C000000000000055
:101020000000000000000000000000000D58020059
:1010300069C000000000000069C0000069C0000035
:10104000755802007B58020069C0000069C00000AA
:1010500069C0000069C0000069C0000069C00000EC
:101060008158020069C0000069C000008758020072
:1010700069C000008D580200935802009958020080
:1010800069C0000069C0000069C0000069C00000BC
:1010900069C0000069C0000069C0000069C00000AC
:1010A00069C000009F58020069C0000069C00000CC
:1010B00069C0000069C0000069C0000069C000008C
:1010C000A558020069C0000069C0000069C00000A6
:1010D00069C0000069C0000069C0000069C000006C
:1010E00069C0000069C0000069C0000069C000005C
:1010F00069C0000069C0000069C0000069C000004C
:1011000069C0000069C0000000F002F824F03FFB55
:101110000AA090E8000C82448344AAF10107DA4552
:1011200001D124F034FBAFF2090EBAE80F0013F03E
:10113000010F18BFFB1A43F001031847584C020077
:10114000784C02000A444FF0000C10F8013B13F0F9
:10115000070408BF10F8014B1D1108BF10F8015B10
:10116000641E05D010F8016B641E01F8016BF9D103
:1011700013F0080F1EBF10F8014BAD1C0C1B09D15A
:101180006D1E58BF01F801CBFAD505E014F8016BCC
:1011900001F8016B6D1EF9D59142D6D3704700005E
:1011A0000023002400250026103A28BF78C1FBD870
:1011B000520728BF30C148BF0B6070471FB500F011
:1011C0003DF88DE80F001FBD1EF0040F0CBFEFF3BC
:1011D0000880EFF30980014A10470000ABBF000010
:1011E000F0B44046494652465B460FB402A0013077
:1011F00001B50648004700BF01BC86460FBC8046CB
:10120000894692469B46F0BC7047000009110000D9
:101210008269034981614FF001001044704700006A
:101220002512000001B41EB400B514F0CBFE01B4C9
:101230000198864601BC01B01EBD000024F0A4BA8E
:1012400070B51A4C054609202070A01C00F0D1F89A
:101250005920A08029462046BDE8704008F0CEB84D
:1012600008F0D7B870B50C461149097829B1A0F13A
:1012700060015E2908D3012013E0602804D06928AA
:1012800002D043F201000CE020CC0A4E94E80E009C
:1012900006EB8000A0F58050241FD0F8806E284611
:1012A000B047206070BD012070470000080000209A
:1012B00018000020F05802003249884201D2012073
:1012C00070470020704770B50446A0F500002E4E10
:1012D000B0F1786F02D23444A4F500042948844266
:1012E00001D2012500E0002500F043F848B125B9FE
:1012F000B44204D32548006808E0012070BD0020F6
:1013000070BD002DF9D1B442F9D321488442F6D200
:10131000F3E710B50446A0F50000B0F1786F03D2F2
:1013200019480444A4F5000400F023F84FF080416C
:1013300030B11648006804E08C4204D2012003E07A
:1013400013488442F8D2002080F0010010BD10B58F
:1013500020B1FFF7DEFF08B1012010BD002010BD55
:1013600010B520B1FFF7AFFF08B1012010BD00207C
:1013700010BD084808490068884201D10120704723
:101380000020704700600200000000201C000020C8
:101390000800002054000020BEBAFECA10B5044662
:1013A0000021012000F03DF800210B2000F039F869
:1013B0000421192000F035F804210D2000F031F847
:1013C00004210E2000F02DF804210F2000F029F850
:1013D0000421C84300F025F80621162000F021F86A
:1013E0000621152000F01DF82046FFF729FF0020F8
:1013F00010BDB62101807047FFF732BF114870471A
:1014000010487047104A10B514680F4B0F4A083344
:101410001A60FFF727FF0C48001D046010BD7047DD
:1014200070474907090E002804DB00F1E02080F82E
:101430000014704700F00F0000F1E02080F8141D48
:101440007047000003F9004210050240010000014E
:10145000FE48002101604160018170472DE9F7439A
:10146000044692B091464068FFF771FF40B1606852
:10147000FFF776FF20B9607800F00300022801D062
:10148000012000E00020F14E30724846FFF71BFFBC
:1014900018B1102015B0BDE8F0834946012001F0D5
:1014A0008EFE0028F6D101258DF842504FF4C05031
:1014B000ADF84000002210A9284606F009FC0028DB
:1014C000E8D18DF842504FF428504FF00008ADF8A5
:1014D000400047461C216846CDF81C8024F0EFF8F8
:1014E0009DF81C0008AA20F00F00401C20F0F0001E
:1014F00010308DF81C0020788DF81D0061789DF863
:101500001E0061F3420040F001008DF81E009DF8BE
:1015100000000AA940F002008DF800002089ADF813
:101520003000ADF83270608907AFADF834000B972A
:10153000606810AC0E900A94684606F0BCF900286A
:10154000A8D1BDF8200030808DF8425042F601202D
:10155000ADF840009DF81E0008AA20F00600801C8F
:1015600020F001008DF81E000220ADF83000ADF82B
:10157000340013A80E900AA9684606F09CF90028CA
:1015800088D1BDF820007080311D484600F033F945
:10159000002887D18DF8425042F6A620ADF84000D1
:1015A0001C216846CDF81C8024F089F89DF81C00A9
:1015B000ADF8345020F00F00401C20F0F000103047
:1015C0008DF81C009DF81D0008AA20F0FF008DF882
:1015D0001D009DF81E000AA920F0060040F0010041
:1015E000801C8DF81E009DF800008DF8445040F0DE
:1015F00002008DF80000CDE90A4711A80E90ADF861
:101600003050684606F057F9002899D1BDF82000FF
:10161000F08000203EE73EB504460820ADF800000B
:101620002046FFF750FE08B110203EBD21460120A4
:1016300001F0C5FD0028F8D12088ADF804006088CD
:10164000ADF80600A088ADF80800E088ADF80A0003
:101650007E4801AB6A468088002106F035FDBDF862
:1016600000100829E1D003203EBD1FB5044600202C
:1016700002900820ADF80800CDF80CD02046FFF706
:1016800022FE10B1102004B010BD704802AA81885B
:101690004FF6FF7006F05AFF0028F4D1BDF808108D
:1016A000082901D00320EEE7BDF800102180BDF825
:1016B00002106180BDF80410A180BDF80610E18021
:1016C000E1E701B582B00220ADF800005F4802AB4F
:1016D0006A464088002106F0F7FCBDF80010022998
:1016E00000D003200EBD1CB5002100910221ADF8F1
:1016F00000100190FFF70DFE08B110201CBD5348EB
:101700006A4641884FF6FF7006F020FFBDF80010D2
:101710000229F3D003201CBDFEB54C4C06461546ED
:10172000207A0F46C00705D00846FFF7CCFD18B158
:101730001020FEBD0F20FEBDF82D01D90C20FEBDEE
:101740003046FFF7C0FD18BB208801A905F0B8FDA1
:101750000028F4D130788DF80500208801A906F022
:1017600091FC0028EBD100909DF800009DF8051039
:1017700040F002008DF80000090703D040F0080097
:101780008DF800002088694606F019FC0028D6D1A3
:10179000ADF8085020883B4602AA002106F094FCD0
:1017A000BDF80810A942CAD00320FEBD7CB505468D
:1017B0000020009001900888ADF800000C462846F3
:1017C0000195FFF7C4FD18B92046FFF7A2FD08B147
:1017D00010207CBD15B1BDF8000050B11B486A4611
:1017E00001884FF6FF7006F0B1FEBDF800102180B1
:1017F0007CBD0C207CBD30B593B0044600200D4666
:101800000090142101A823F05AFF1C2108A823F0FE
:1018100056FF9DF80000CDF808D020F00F00401CC6
:1018200020F0F00010308DF800009DF8010020F04D
:10183000FF008DF801009DF8200040F002008DF8B7
:10184000200001208DF8460002E000002002002068
:1018500042F60420ADF8440011A801902088ADF8AC
:101860003C006088ADF83E00A088ADF84000E088FC
:10187000ADF842009DF8020006AA20F00600801C88
:1018800020F001008DF802000820ADF80C00ADF842
:1018900010000FA8059001A908A806F00CF8002870
:1018A00003D1BDF818002880002013B030BD00001F
:1018B000F0B5007B059F1E4614460D46012800D05A
:1018C000FFDF0C2030803A203880002C08D0287AA6
:1018D000032806D0287B012800D0FFDF1720608175
:1018E000F0BDA889FBE72DE9F04786B0144691F8D2
:1018F0000C900E9A0D46B9F1010F0BD01021007B10
:101900002E8A8846052807D0062833D0FFDF06B088
:10191000BDE8F0870221F2E7E8890C2100EB4000E6
:1019200001EB4000188033201080002CEFD0E889B4
:10193000608100271AE00096688808F1020301AA76
:10194000696900F084FF06EB0800801C07EB470183
:1019500086B204EB4102BDF8040090810DF106014E
:1019600040460E3212F0D3FD7F1CBFB26089B842F0
:10197000E1D8CCE734201080E889B9F1010F11D00B
:10198000122148430E301880002CC0D0E8896081B5
:101990004846B9F1010F00D00220207300270DF155
:1019A000040A1FE00621ECE70096688808F10203AC
:1019B00001AA696900F04BFF06EB0800801C86B2A3
:1019C000B9F1010F12D007EBC70004EB4000BDF8DE
:1019D0000410C18110220AF10201103023F0CEFD63
:1019E0007F1CBFB26089B842DED890E707EB4701A1
:1019F00004EB4102BDF80400D0810AF10201404627
:101A0000103212F084FDEBE72DE9F0470E4688B066
:101A100090F80CC096F80C80378AF5890C20109944
:101A200002F10C044FF0000ABCF1030F08D0BCF126
:101A3000040F3ED0BCF1070F7DD0FFDF08B067E791
:101A400005EB850C00EB4C00188031200880002A43
:101A5000F4D0A8F1060000F0FF09558125E0182117
:101A600001A823F02CFE00977088434601AA7169F3
:101A700000F0EDFEBDF804002080BDF80600E08017
:101A8000BDF808002081A21C0DF10A01484612F0A1
:101A90003EFDB9F1000F00D018B184F804A0A4F8FD
:101AA00002A007EB080087B20A346D1EADB2D6D291
:101AB000C4E705EB850C00EB4C0018803220088051
:101AC000002ABBD0A8F1050000F0FF09558137E0DE
:101AD00000977088434601AA716900F0B8FE9DF82E
:101AE0000600BDF80410E1802179420860F300018E
:101AF00062F34101820862F38201C20862F3C3010A
:101B0000020962F30411420962F34511820962F38A
:101B100086112171C0096071BDF80700208122463D
:101B20000DF10901484612F0F2FC18B184F802A048
:101B3000A4F800A000E007E007EB080087B20A3431
:101B40006D1EADB2C4D279E7A8F1020084B205FBE4
:101B500008F000F10E0CA3F800C035230B80002A1A
:101B6000A6D055819481009783B270880E32716936
:101B700000F06DFE62E72DE9F84F1E460A9D0C4607
:101B800081462AB1607A00F58070D080E0891081AA
:101B900099F80C000C274FF000084FF00E0A0D28A2
:101BA00073D2DFE800F09E070E1C28303846556AD5
:101BB00073737300214648460095FFF779FEBDE830
:101BC000F88F207B9146082802D0032800D0FFDF41
:101BD000378030200AE000BFA9F80A80EFE7207BB9
:101BE0009146042800D0FFDF378031202880B9F1EA
:101BF000000FF1D1E3E7207B9146042800D0FFDFFE
:101C000037803220F2E7207B9146022800D0FFDFA8
:101C100037803320EAE7207B1746022800D0FFDF19
:101C20003420A6F800A02880002FC8D0A7F80A808A
:101C3000C5E7207B1746042800D0FFDF3520A6F833
:101C400000A02880002FBAD04046A7F80A8012E0F2
:101C5000207B1746052802D0062800D0FFDF102081
:101C6000308036202880002FA9D0E0897881A7F81D
:101C70000E80B9F80E00B881A1E7207B91460728B5
:101C800000D0FFDF37803720B0E72AE04FF01200A6
:101C900018804FF038001700288090D0E0897881B4
:101CA000A7F80E80A7F8108099F80C000A2805D034
:101CB0000B2809D00C280DD0FFDF80E7207B0A28F5
:101CC00000D0FFDF01200AE0207B0B2800D0FFDFDF
:101CD000042004E0207B0C2800D0FFDF05203873AF
:101CE0006DE7FFDF6BE770B50C46054601F0ABFB17
:101CF00020B10078222804D2082070BD43F20200EF
:101D000070BD0521284610F075FE206008B1002046
:101D100070BD032070BD30B44880087820F00F00FB
:101D2000C01C20F0F000903001F8080B1DCA81E8BB
:101D30001D0030BC07F0E3BB2DE9FF4784B000274E
:101D40008246029707989046894612300AF0DCF9DD
:101D5000401D20F00306079828B907A95046FFF751
:101D6000C2FF002854D1B9F1000F05D00798017BBC
:101D700019BB052504681BE098F80000092803D06A
:101D80000D2812D0FFDF46E0079903254868B0B35D
:101D9000497B42887143914239D98AB2B3B2011D5D
:101DA00010F09BFC0446078002E0079C04250834E1
:101DB0000CB1208810B1032D29D02CE00798012107
:101DC00012300AF0D3F9ADF80C00024602AB2946F6
:101DD000504608F000FA070001D1A01C02900798B5
:101DE0003A461230C8F80400A8F802A003A94046F9
:101DF000029B0AF0C8F9D8B10A2817D200E006E021
:101E0000DFE800F007091414100B0D14141213204E
:101E100014E6002012E6112010E608200EE643F238
:101E200003000BE6072009E60D2007E6032005E680
:101E3000BDF80C002346CDE900702A4650460799AC
:101E400000F015FD57B9032D08D10798B3B2417BB7
:101E5000406871438AB2011D10F053FCB9F1000FC4
:101E6000D7D0079981F80C90D3E72DE9FE4F914622
:101E70001A881C468A468046FAB102AB494608F0E9
:101E8000AAF9050019D04046A61C278810F0F6FED6
:101E90003246072629463B46009610F004FB208870
:101EA0002346CDE900504A465146404600F0DFFC4B
:101EB000002020800120BDE8FE8F0020FBE710B548
:101EC00086B01C46AAB104238DF800301388ADF803
:101ED00008305288ADF80A208A788DF80E200988DB
:101EE000ADF80C1000236A462146FFF725FF06B027
:101EF00010BD1020FBE770B50D46052110F07AFDEE
:101F0000040000D1FFDF294604F11200BDE8704053
:101F10000AF015B92DE9F8430D468046002607F072
:101F2000EBFA04462878102878D2DFE800F0773BF7
:101F30003453313112313131083131313131287975
:101F4000001FC0B2022801D0102810D114BBFFDF3F
:101F500035E004B9FFDF0521404610F04BFD007B62
:101F6000032806D004280BD0072828D0FFDF072637
:101F700055E02879801FC0B2022820D050B1F6E782
:101F80002879401FC0B2022819D0102817D0EEE7D8
:101F900004B9FFDF13E004B9FFDF287901280ED16F
:101FA000172137E00521404610F024FD070000D13D
:101FB000FFDF07F1120140460AF09EF82CB12A46D5
:101FC00021464046FFF7A7FE29E01321404602F0D4
:101FD000F7FC24E004B9FFDF0521404610F00AFDBC
:101FE000060000D1FFDF694606F112000AF08EF804
:101FF000060000D0FFDFA988172901D2172200E0D0
:102000000A46BDF80000824202D9014602E005E01E
:102010001729C5D3404600F03AFCD0E7FFDF304631
:10202000BDE8F883401D20F0030219B102FB01F066
:10203000001D00E000201044704713B5009848B11F
:102040000024684610F0F3FA002C02D1F74A0099F8
:1020500011601CBD01240020F4E72DE9F0470C4677
:1020600015462421204623F02AFB05B9FFDFA87876
:1020700060732888DFF8B4A3401D20F00301AF7817
:102080008946DAF8000010F0F0FA060000D1FFDF10
:102090004FF000082660A6F8008077B109FB07F131
:1020A000091D0AD0DAF8000010F0DFFA060000D1AE
:1020B000FFDF6660C6F8008001E0C4F8048029886C
:1020C00004F11200BDE8F0470AF008B82DE9F04726
:1020D000804601F112000D4681460AF015F8401DB8
:1020E000D24F20F003026E7B14462968386810F046
:1020F000E7FA3EB104FB06F2121D03D069683868A6
:1021000010F0DEFA052010F01DFC0446052010F04A
:1021100021FC201A012802D1386810F09BFA4946A8
:102120004046BDE8F04709F0EEBF70B50546052111
:1021300010F060FC040000D1FFDF04F1120128461A
:10214000BDE8704009F0D8BF2DE9F04F91B04FF0D5
:10215000000BADF834B0ADF804B047880C46054626
:1021600092460521384610F045FC060000D1FFDFFD
:1021700024B1A780A4F806B0A4F808B029780922F1
:102180000B20B2EB111F7DD12A7A04F11001382700
:102190004FF00C084FF001090391102A73D2DFE8C9
:1021A00002F072F2F1F07F08D2888D9F3DDBF3EEF2
:1021B000B6B6307B022800D0FFDFA88908EBC0014B
:1021C000ADF804103021ADF83410002C25D060811A
:1021D000B5F80E9000271DE004EBC708317C88F8A5
:1021E0000E10F189A8F80C10CDF80090688804232F
:1021F00004AA296900F02BFBBDF81010A8F81010F4
:1022000009F10400BDF812107F1C1FFA80F9A8F82C
:102210001210BFB26089B842DED80DE1307B0228CF
:1022200000D0FFDFE98908EBC100ADF804003020E1
:10223000ADF83400287B0A90001FC0B20F90002C2C
:10224000EBD06181B5F81090002725E0CDF8009023
:102250006888696903AA0A9B00F0F9FA0A9804EBF6
:10226000C70848441FFA80F908F10C0204A90F9826
:1022700012F04DF918B188F80EB0A8F80CB0BDF8FE
:102280000C1001E0D4E0CFE0A8F81010BDF80E105B
:102290007F1CA8F81210BFB26089B842D6D8CBE034
:1022A0000DA8009001AB224629463046FFF71BFBE4
:1022B000C2E0307B082805D0FFDF03E0307B082830
:1022C00000D0FFDFE8891030ADF804003620ADF80B
:1022D0003400002C3FD0A9896181F189A18127E0D8
:1022E000307B092800D0FFDFA88900F10C01ADF890
:1022F00004103721ADF83410002C2CD06081E8890F
:102300000090AB89688804F10C02296956E0E889DD
:102310003921103080B2ADF80400ADF83410002C33
:1023200074D0A9896181287A0E280AD002212173EC
:10233000E989E181288A0090EB8968886969039AB4
:102340003CE00121F3E70DA8009001AB22462946AD
:102350003046FFF759FB6FE0307B0A2800D0FFDFE3
:102360001220ADF80400ADF834704CB3A989618136
:10237000A4F810B0A4F80EB084F80C905CE020E053
:1023800002E031E039E042E0307B0B2800D0FFDF93
:10239000288AADF834701230ADF8040084B10421FD
:1023A0002173A9896181E989E181298A2182688A69
:1023B00000902B8A688804F11202696900F047FADC
:1023C0003AE0307B0C2800D0FFDF1220ADF804008B
:1023D000ADF834703CB305212173A4F80AB0A4F819
:1023E0000EB0A4F810B027E00DA8009001AB224673
:1023F00029463046FFF75CFA1EE00DA8009001ABBD
:10240000224629463046FFF7B6FB15E034E03B2173
:10241000ADF80400ADF8341074B3A4F80690A4F835
:1024200008B084F80AB007E0FFDF05E010000020E4
:10243000297A012917D0FFDFBDF80400AAF80000AF
:102440006CB1BDF834002080BDF804006080BDF898
:102450003400392803D03C2801D086F80CB011B0E4
:102460000020BDE8F08F3C21ADF80400ADF8341039
:1024700014B1697AA172DFE7AAF80000EFE72DE94D
:10248000F84356880F46804615460521304610F021
:10249000B1FA040000D1FFDF123400943B464146FC
:1024A00030466A6809F0A3FFBAE570B50D4605210C
:1024B00010F0A0FA040000D1FFDF294604F1120059
:1024C000BDE8704009F02DBE70B50D46052110F035
:1024D00091FA040000D1FFDF294604F11200BDE8A3
:1024E000704009F04BBE70B50546052110F082FA28
:1024F000040000D1FFDF04F1080321462846BDE8AF
:1025000070400422B1E470B50546052110F072FA5E
:10251000040000D1FFDF214628462368BDE8704053
:102520000522A2E470B50646052110F063FA040006
:1025300000D1FFDF04F1120009F0E6FD401D20F09C
:10254000030511E0011D008803224318214630468F
:10255000FFF78BFC00280BD0607BABB2684382B2E4
:102560006068011D10F003F9606841880029E9D115
:1025700070BD70B50E46054606F0BEFF040000D1E2
:10258000FFDF0120207266726580207820F00F0046
:10259000C01C20F0F00030302070BDE8704006F024
:1025A000AEBF2DE9F0438BB00D461446814606A917
:1025B000FFF799FB002814D14FF6FF7601274FF45F
:1025C00020588CB103208DF800001020ADF81000C9
:1025D00007A8059007AA204604A911F0B7FF78B113
:1025E00007200BB0BDE8F0830820ADF808508DF847
:1025F0000E708DF80000ADF80A60ADF80C800CE0AC
:102600000698A17801742188C1818DF80E70ADF80B
:102610000850ADF80C80ADF80A606A4602214846C1
:10262000069BFFF789FBDCE708B501228DF8022045
:1026300042F60202ADF800200A4603236946FFF77E
:102640003EFC08BD08B501228DF8022042F60302C7
:10265000ADF800200A4604236946FFF730FC08BDA8
:1026600000B587B079B102228DF800200A88ADF854
:1026700008204988ADF80A1000236A460521FFF7B3
:102680005BFB07B000BD1020FBE709B1072316E490
:102690000720704770B588B00D461446064606A957
:1026A000FFF721FB00280ED17CB10620ADF80850C1
:1026B0008DF80000ADF80A40069B6A460821DC81CF
:1026C0003046FFF739FB08B070BD05208DF80000DB
:1026D000ADF80850F0E700B587B059B107238DF881
:1026E0000030ADF80820039100236A460921FFF766
:1026F00023FBC6E71020C4E770B588B00C46064639
:10270000002506A9FFF7EFFA0028DCD10698012181
:10271000123009F02BFD9CB12178062921D2DFE887
:1027200001F0200505160318801E80B2C01EE28845
:1027300080B20AB1A3681BB1824203D90C20C2E760
:102740001020C0E7042904D0A08850B901E0062079
:10275000B9E7012913D0022905D004291CD0052985
:102760002AD00720AFE709208DF800006088ADF877
:102770000800E088ADF80A00A068039023E00A2072
:102780008DF800006088ADF80800E088ADF80A0018
:10279000A0680A25039016E00B208DF800006088E1
:1027A000ADF80800A088ADF80A00E088ADF80C008C
:1027B000A0680B25049006E00C208DF800006078DE
:1027C0008DF808000C256A4629463046069BFFF71F
:1027D000B3FA78E700B587B00D228DF80020ADF888
:1027E000081000236A461946FFF7A6FA49E700B524
:1027F00087B071B102228DF800200A88ADF8082058
:102800004988ADF80A1000236A460621FFF794FABA
:1028100037E7102035E770B586B0064601200D4633
:10282000ADF808108DF80000014600236A463046D6
:10283000FFF782FA040008D12946304605F05EFC15
:102840000021304605F078FC204606B070BDF8B592
:102850001C4615460E46069F10F0FEF92346FF1D46
:10286000BCB231462A4600940FF0E9FDF8BD30B401
:102870001146DDE902423CB1032903D0002330BCFC
:1028800008F034BB0123FAE71A8030BC704770B5FA
:102890000C460546FFF72FFB2146284605F03DFC78
:1028A0002846BDE87040012105F046BC4FF0E0220B
:1028B0004FF400400021C2F88001BFF34F8FBFF3F7
:1028C0006F8F1748016001601649900208607047D9
:1028D000134900B500220A600A60124B4FF0607283
:1028E0001A60002808BF00BD0F4A104BDFF840C037
:1028F00001280CD002281CBFFFDF00BD03200860A8
:102900001A604FF4000000BFCCF8000000BD0220A8
:1029100008601A604FF04070F6E700B5FFDF00BDB9
:1029200000F5004008F50140A002002014F5004029
:1029300004F5014070B50B2000F0BDF9082000F04F
:10294000BAF900210B2000F0D4F90021082000F092
:10295000D0F9F44C01256560A5600020C4F8400161
:10296000C4F84401C4F848010B2000F0B5F9082070
:1029700000F0B2F90B2000F091F9256070BD10B5A0
:102980000B2000F098F9082000F095F9E5480121A6
:1029900041608160E4490A68002AFCD10021C0F846
:1029A0004011C0F84411C0F848110B2000F094F910
:1029B000BDE81040082000F08FB910B50B2000F0E2
:1029C0008BF9BDE81040082000F086B900B530B1A1
:1029D000012806D0022806D0FFDF002000BDD34822
:1029E00000BDD34800BDD248001D00BD70B5D1491F
:1029F0004FF000400860D04DC00BC5F80803CF4829
:102A000000240460C5F840410820C43500F053F9A3
:102A1000C5F83C41CA48047070BD08B5C14A0021E0
:102A200028B1012811D002281CD0FFDF08BD4FF4C7
:102A30008030C2F80803C2F84803BB483C3001604C
:102A4000C2F84011BDE80840D0E74FF40030C2F8AA
:102A50000803C2F84803B44840300160C2F844118A
:102A6000B3480CE04FF48020C2F80803C2F84803D2
:102A7000AD4844300160C2F84811AD48001D0068FF
:102A8000009008BD70B516460D460446022800D9D0
:102A9000FFDF0022A348012304F110018B4000EB6B
:102AA0008401C1F8405526B1C1F84021C0F8043373
:102AB00003E0C0F80833C1F84021C0F8443370BDCA
:102AC0002DE9F0411D46144630B1012833D00228CB
:102AD00038D0FFDFBDE8F081891E002221F07F4160
:102AE0001046FFF7CFFF012D23D00020944D924FC9
:102AF000012668703E61914900203C39086002203F
:102B0000091D08608D490420303908608B483D3428
:102B1000046008206C6000F0DFF83004C7F804039C
:102B2000082000F0BBF88349F007091F08602E70E9
:102B3000D0E70120DAE7012B02D00022012005E0D6
:102B40000122FBE7012B04D000220220BDE8F04166
:102B500098E70122F9E774480068704770B500F003
:102B6000D8F8704C0546D4F840010026012809D158
:102B7000D4F80803C00305D54FF48030C4F8080327
:102B8000C4F84061D4F8440101280CD1D4F80803FA
:102B9000800308D54FF40030C4F80803C4F844613A
:102BA000012012F0A9FCD4F8480101280CD1D4F876
:102BB0000803400308D54FF48020C4F80803C4F884
:102BC0004861022012F098FC5E48056070BD70B547
:102BD00000F09FF85A4D0446287850B1FFF706FFE1
:102BE000687818B10020687012F086FC55480460BF
:102BF00070BD0320F8E74FF0E0214FF40010C1F85A
:102C000000027047152000F067B84B4901200861A9
:102C1000082000F061B848494FF47C10C1F808035F
:102C20000020024601EB8003C3F84025C3F8402191
:102C3000401CC0B20628F5D37047410A43F609523A
:102C40005143C0F3080010FB02F000F5807001EB67
:102C50005020704710B5430B48F2376463431B0C98
:102C60005C020C60384C03FB0400384B4CF2F72438
:102C700043435B0D13FB04F404EB402000F580702C
:102C80004012107008681844086010BD2C48406855
:102C9000704729490120C1F800027047002809DB6C
:102CA00000F01F02012191404009800000F1E02066
:102CB000C0F80011704700280DDB00F01F02012151
:102CC00091404009800000F1E020C0F88011BFF37E
:102CD0004F8FBFF36F8F7047002809DB00F01F0292
:102CE000012191404009800000F1E020C0F88012ED
:102CF00070474907090E002804DB00F1E02080F846
:102D00000014704700F00F0000F1E02080F8141D5F
:102D100070470C48001F00680A4A0D49121D1160D7
:102D20007047000000B0004004B500404081004002
:102D300044B1004008F5014000800040408500405B
:102D40003400002014050240F7C2FFFF6F0C0100A1
:102D5000010000010A4810B5046809490948083112
:102D6000086012F05DFC0648001D046010BD0649B5
:102D7000002008604FF0E0210220C1F88002704777
:102D80001005024001000001FC1F004010B50D209D
:102D900000F077F8C4B26FF0040000F072F8C0B22F
:102DA000844200D0FFDF3E490120086010BD70B5AD
:102DB0000D2000F048F83B4C0020C4F8000101252C
:102DC000C4F804530D2000F04FF825604FF0E021C7
:102DD0006014C1F8000170BD10B50D2000F033F88B
:102DE0003048012141600021C0F80011BDE81040C9
:102DF0000D2000F039B82C4810B504682A492B483A
:102E0000083108602749D1F80001012804D0FFDF0C
:102E10002548001D046010BD2148001D00680022E7
:102E2000C0B2C1F8002113F047F8F1E710B51D4812
:102E3000D0F800110029FBD0FFF7DDFFBDE81040FE
:102E40000D2000F011B800280DDB00F01F02012159
:102E500091404009800000F1E020C0F88011BFF3EC
:102E60004F8FBFF36F8F7047002809DB00F01F0200
:102E7000012191404009800000F1E020C0F880125B
:102E80007047002804DB00F1E02090F8000405E022
:102E900000F00F0000F1E02090F8140D4009704799
:102EA00004D5004000D000401005024001000001A0
:102EB0004FF0E0214FF00070C1F8800101F5C071C2
:102EC000BFF34F8FBFF36F8FC1F80001384B8022E3
:102ED00083F8002441F8800C704700B502460420B6
:102EE000344903E001EBC0031B792BB1401EC0B293
:102EF000F8D2FFDFFF2000BD41F8302001EBC00118
:102F000000224A718A7101220A7100BD294A0021FA
:102F100002EBC0000171704710B50446042800D3CD
:102F2000FFDF244800EBC4042079012800D0FFDF34
:102F30006079A179401CC0B2814200D060714FF02D
:102F4000E0214FF00070C1F8000210BD2DE9F04102
:102F500019480568184919480831086014480426BA
:102F600090F80004134F4009154C042818D0FFDFD7
:102F700016E0217807EBC1000279012A08D14279D5
:102F800083799A4204D04279827157F831008047A0
:102F90002078401CC0B22070042801D3002020708B
:102FA000761EF6B2E5D20448001D0560BDE8F0814A
:102FB00019E000E0D80500201005024001000001E2
:102FC000500000200548064A0168914201D10021C5
:102FD000016004490120086070470000540000208F
:102FE000BEBAFECA40E5014070B50C46054609F080
:102FF0009BFB21462846BDE870400AF080BC704724
:103000002CFFFFFFDBE5B15100600200B600FFFFBF
:103010008C00000069915B00935FFEEDA0843C731F
:10302000F87462145E06C0CB72F2136030B5F84DCE
:103030000446062CA9780ED2DFE804F0030E0E0E2B
:103040000509FFDF08E0022906D0FFDF04E00329BD
:1030500002D0FFDF00E0FFDFAC7030BD30B50446CA
:103060001038EB4D07280CD2DFE800F0040C060CFA
:103070000C0C0C00FFDF05E0287E112802D0FFDFDA
:1030800000E0FFDF2C7630BD2DE9F04111F0C8FBE8
:10309000044612F0A1FD201AC5B206200FF052FC22
:1030A000044606200FF056FC211AD94C207E122827
:1030B00018D000200F1807200FF044FC0646072008
:1030C0000FF048FC301A3918207E13280CD000204D
:1030D0000144A078042809D000200844281AC0B26E
:1030E000BDE8F0810120E5E70120F1E70120F4E7E8
:1030F000C74810B590F825004108C54800F12600E2
:1031000005D00DF018FBBDE8104006F00BB80DF02F
:10311000F3FAF8E730B50446A1F120000D460A287D
:103120004AD2DFE800F005070C1C2328353A3F445B
:10313000FFDF42E0207820283FD1FFDF3DE0B448A8
:103140008178052939D0007E122836D020782428AD
:1031500033D0252831D023282FD0FFDF2DE0207851
:1031600022282AD0232828D8FFDF26E0207822280A
:1031700023D0FFDF21E0207822281ED024281CD075
:1031800026281AD0272818D0292816D0FFDF14E0C7
:103190002078252811D0FFDF0FE0207825280CD0DB
:1031A000FFDF0AE02078252807D0FFDF05E0207840
:1031B000282802D0FFDF00E0FFDF257030BD1FB5FB
:1031C00004466A46002001F03CFEB4B1BDF802207E
:1031D0004FF6FF700621824201D1ADF80210BDF812
:1031E0000420824201D1ADF80410BDF808108142DC
:1031F00003D14FF44860ADF8080068460EF014F9AA
:1032000005F090FF04B010BD70B514460D4606469B
:10321000FEF759F858B90DB1A54201D90C2070BD7F
:10322000002408E056F82400FEF74DF808B11020FD
:1032300070BD641CE4B2AC42F4D3002070BD2DE933
:10324000F04105461F4690460E4600240068FEF7F2
:1032500087F830B9A98828680844401EFEF780F82E
:1032600008B110203CE728680028A88802D0B8429E
:1032700002D850E00028F5D0092031E72968085D20
:10328000B8B1671CCA5D152A2ED03CDC152A3AD28B
:10329000DFE802F03912222228282A2A313139396E
:1032A00039393939393939392200085D30BB641C64
:1032B000A4B2A242F9D833E00228DDD1A01C085CF8
:1032C00088F80000072801D2400701D40A2007E748
:1032D000307840F0010015E0C143C90707E001283C
:1032E00007D010E00620FBE60107A1F1805100297C
:1032F000F5D01846F4E63078810701D50B20EFE6CB
:1033000040F0020030702868005D384484B2A8881C
:10331000A04202D2B0E74FF4485382B2A242ADD8E5
:103320000020DDE610B5027843F2022354080122A2
:10333000022C12D003DC3CB1012C16D106E0032C88
:1033400010D07F2C11D112E0002011E080790324ED
:10335000B4EB901F09D10A700BE08079B2EB901F9B
:1033600003D1F8E780798009F5D0184610BDFF2019
:103370000870002010BD08B500208DF8000024481A
:1033800090F82E1049B190F82F0002280ED0032893
:103390000ED0FFDF9DF8000008BD1D4869462530AE
:1033A00001F09EFD0028F5D0FFDFF3E7032000E0E9
:1033B00001208DF80000EDE738B50C46054669465A
:1033C00001F08EFD00280DD19DF80010207861F3EA
:1033D0004700207055F8010FC4F80100A888A4F830
:1033E0000500002038BD38B51378A8B1022813D0E5
:1033F000FF281AD007A46D46246800944C7905EB89
:103400009414247864F347031370032809D00FE061
:10341000EC0100200302FF0123F0FE0313700228D9
:10342000F3D1D8B240F0010005E043F0FE00107087
:10343000107820F0010010700868C2F80100888838
:10344000A2F8050038BD02210FF0D4BA38B50C46F9
:103450000978222901D2082038BDADF800008DF886
:10346000022068460DF0A9F905F05CFE050003D1C5
:1034700021212046FFF74EFE284638BD1CB500200E
:103480008DF80000CDF80100ADF80500FB4890F87C
:103490002E00022801D0012000E000208DF8070056
:1034A00068460DF0FAFA002800D0FFDF1CBD0022AC
:1034B0000A80437892B263F3451222F040020A80F8
:1034C00000780C282BD2DFE800F02A06090E11162E
:1034D000191C1F220C2742F0110009E042F01D00C8
:1034E00008800020704742F0110012E042F0100006
:1034F00040F00200F4E742F01000F1E742F0010072
:10350000EEE742F0010004E042F00200E8E742F09A
:10351000020040F00400E3E742F00400E0E7072087
:1035200070472DE9FF478AB00025BDF82C60824620
:103530001C4691468DF81C50700703D56068FDF756
:10354000C2FE68B9CD4F4FF0010897F82E0058B170
:1035500097F82F00022807D16068FDF701FF18B126
:1035600010200EB0BDE8F087300702D5A089802872
:103570003ED8700705D4B9F1000F02D097F82400A7
:10358000A0B3E07DC0F300108DF81B00627D072022
:10359000032162B3012A2DD0022AE2D0042AE0D10D
:1035A0008DF81710F00628D4A27D07202AB3012A2F
:1035B00023D0022A24D0042AD3D18DF8191000BFB9
:1035C0008DF81590606810B307A9FFF7ABFE0028CF
:1035D000C7D19DF81C00FF2816D0606850F8011F65
:1035E000CDF80F108088ADF8130014E000E001E082
:1035F0000720B6E78DF81780D4E78DF81980DFE74C
:1036000002208DF81900DBE743F20220A9E7CDF88C
:103610000F50ADF81350E07B40B9207C30B9607C8E
:1036200020B9A07C10B9E07CC00601D0062098E744
:103630008DF800A0BDF82C00ADF80200A068019044
:10364000A068029004F10F0001F03EFC8DF80C0020
:10365000FFF791FE8DF80D009DF81C008DF80E000F
:103660008DF816508DF81850E07D08A900F00F0075
:103670008DF81A0068460EF015F805F053FD70E756
:10368000F0B58FB000258DF830508DF814508DF8BE
:10369000345006468DF828500195029503950495FF
:1036A00019B10FC901AC84E80F00744CA07805284B
:1036B00001D004280CD101986168884200D120B95A
:1036C0000398E168884203D110B108200FB0F0BD23
:1036D000207DC00601D51F2700E0FF273B460DAA2D
:1036E00005A903A8FFF7ABFD0028EFD1A08AC10709
:1036F00002D0C00600D4EE273B460AAA0CA901A8B6
:10370000FFF79DFD0028E1D19DF81400C00701D00E
:103710000A20DBE7A08A410708D4A17D31B19DF8DA
:103720002810890702D043F20120CFE79DF8281026
:10373000C90709D0400707D4208818B144F2506166
:10374000884201D90720C1E78DF818508DF819601B
:10375000BDF80800ADF81A000198079006A80DF012
:10376000BBFF05F0DFFC0028B0D18DF820508DF8AC
:103770002160BDF81000ADF822000398099008A858
:103780000DF0C9FF05F0CEFC00289FD101AD241D2E
:1037900095E80F0084E80F00002097E770B586B029
:1037A0000D46040005D0FDF7DBFD20B1102006B06A
:1037B00070BD0820FBE72078C107A98802D0FF2947
:1037C00002D303E01F2901D20920F0E7800763D468
:1037D000FFF75AFC38B12178C1F3C100012804D0A9
:1037E000032802D005E01320E1E7244890F82400E4
:1037F000C8B1C8074FF001064FF0000502D08DF8A0
:103800000F6001E08DF80F50FFF7B5FD8DF8000057
:1038100020786946C0F3C1008DF8010060788DF80A
:103820000250C20801D00720C1E730B3C20701D05F
:103830008DF80260820705D59DF8022042F0020251
:103840008DF80220400705D59DF8020040F00400E5
:103850008DF80200002022780B18C2F38002DA7083
:1038600001EB40026388D380401CA388C0B253811F
:103870000228F0D3207A78B905E001E0EC010020BD
:103880008DF80260E6E7607A30B9A07A20B9E07A74
:1038900010B9207BC00601D0062088E704F108009B
:1038A00001F012FB8DF80E0068460DF0BFFA05F02E
:1038B00039FC002889D18DF810608DF81150E0880E
:1038C000ADF81200ADF8145004A80DF002FB05F09D
:1038D00029FC002888D12078C00701D0152000E0FD
:1038E0001320FFF7BBFB002061E72DE9FF47022013
:1038F000FB4E8DF804000027708EADF80600B84628
:1039000043F202094CE001A80EF0DBFF050006D0EF
:10391000708EA8B3A6F83280ADF806803EE0039C16
:10392000A07F01072DD504F124000090A28EBDF8E0
:103930000800214604F1360301F05FFC050005D0C4
:103940004D452AD0112D3CD0FFDF3AE0A07F20F07A
:103950000801E07F420862F3C711A177810861F393
:103960000000E07794F8210000F01F0084F82000A8
:103970002078282826D129212046FFF7CBFB21E0FB
:1039800014E040070AD5BDF8080004F10E0101F06B
:10399000B1FA05000DD04D4510D100257F1CFFB2B6
:1039A00002200EF0CFFF401CB842ACD8052D11D03C
:1039B00008E0A07F20F00400A07703E0112D00D0E4
:1039C000FFDF0025BDF806007086052D04D02846CF
:1039D00004B0C7E5A6F832800020F9E770B50646C6
:1039E000FFF731FD054605F087FD040000D1FFDF3C
:1039F0006680207820F00F00801C20F0F00020303E
:103A000020700320207295F83E006072BDE870407F
:103A100005F075BD2DE9F04786B0040000D1FFDF49
:103A20002078AF4D20F00F00801C20F0F0007030A7
:103A3000207060680178491F1B2933D2DFE801F04C
:103A4000FE32323255FD320EFDFD42FC323232780A
:103A5000FCFCFBFA3232FCFCF9F8FC00C68830466C
:103A6000FFF7F1FC0546304607F03EF9E0B160682B
:103A7000007A85F83E0021212846FFF74BFB3046AF
:103A8000FEF753FB304603F05BFE3146012012F097
:103A9000D3FCA87F20F01000A877FFF726FF0028AE
:103AA00000D0FFDF06B05DE5207820F0F000203088
:103AB00020700320207266806068007A607205F0D2
:103AC0001EFDD8E7C5882846FFF7BDFC00B9FFDF1B
:103AD00060680079012800D0FFDF6068017A06B0D5
:103AE0002846BDE8F04707F0DEBCC6883046FFF741
:103AF000AAFC050000D1FFDF05F001FD606831463A
:103B00000089288160684089688160688089A8810F
:103B1000012012F091FC0020A875A87F00F003009E
:103B20000228BFD1FFF7E1FE0028BBD0FFDFB9E7D5
:103B300000790228B6D000B1FFDF05F0E0FC66682E
:103B4000B6F806A0307A361D012806D0687E814678
:103B500005F054FA070003D101E0E878F7E7FFDF4A
:103B60000022022150460EF03CFF040000D1FFDF8E
:103B700022212046FFF7CEFA3079012800D002201A
:103B8000A17F804668F30101A177308B2081708B83
:103B90006081B08BA08184F822908DF80880B8688D
:103BA0000090F86801906A46032150460EF019FF14
:103BB00000B9FFDFB888ADF81000B8788DF81200B2
:103BC00004AA052150460EF00CFF00B9FFDFB888AB
:103BD000ADF80C00F8788DF80E0003AA04215046C9
:103BE0000EF0FFFE00B9FFDF062106F1120001F022
:103BF0009FF940B37079800700D5FFDF7179E07DD0
:103C000061F34700E075D6F80600A0617089A083D3
:103C1000062106F10C0001F08BF9F0B195F82500B2
:103C20004108607861F347006070D5F8260006E02F
:103C30003EE036E06DE055E04AE02CE040E0C4F8BC
:103C40000200688D12E0E07D20F0FE00801CE0752F
:103C5000D6F81200A061F08AD9E7607820F0FE0063
:103C6000801C6070F068C4F80200308AE080B8F10F
:103C7000010F04D0B8F1020F05D0FFDF12E70320D7
:103C8000FFF7D4F90EE7287E122800D0FFDF1120BD
:103C9000FFF7E4F906E706B02046BDE8F04701F07B
:103CA00035BD05F02CFC15F8300F40F0020005E0A2
:103CB00005F025FC15F8300F40F004002870F1E6FF
:103CC000287E132809D01528D8D11620FFF7C6F969
:103CD00006B0BDE8F04705F012BC1420F6E700007E
:103CE000EC010020A978052909D00429C6D105F0E6
:103CF00006FC022006B0BDE8F047FFF797B900794F
:103D00000028BBD0E87801F0C6F805F0F8FB0320E6
:103D1000F0E7287E122802D1687E01F0BCF811205D
:103D2000D4E72DE9F047054600784FF00008000978
:103D3000DFF8C0A891460C464646012875D00228F7
:103D400074D007280AD00A2871D0FFDFA9F80060D4
:103D500014B1A4F800806680002003E4696801279C
:103D600004F108000A784FF0020C4FF6FF73172A8F
:103D70007ED00EDC142A32D006DC052A68D0092A4F
:103D800010D0102A75D120E0152A73D0162AF9D147
:103D9000F8E0183A082A6CD2DFE802F0F36B6B0AFD
:103DA000CAF2DFF1C8884FF01208102621468DE1D3
:103DB0004FF01C080A26BCB38888A0806868807908
:103DC00020726868C0796072C0E74FF01B08142643
:103DD00054B30320207268688088A080B6E70A790F
:103DE0003C2AB3D00D1D4FF010082C26E4B1698891
:103DF000A180298B6182298B2182698BA182A98B69
:103E0000E1826B790246A91D1846FFF7ECFA297981
:103E1000002001290CD084F80FC0FF212176E06139
:103E200020626062A06291E70FE02EE151E18CE137
:103E3000E77320760AF1040090E80E00DAF810002B
:103E4000C4E90930C4E9071280E7A9F8006083E7F4
:103E50002C264FF01D08002CF7D00546A380887B48
:103E60002A880F1D60F300022A80887B400802E048
:103E70009DE007E1BEE060F341022A80887B800874
:103E800060F382022A80887BB91CC00860F3C302F9
:103E90002A80B87A0011401C60F3041202F07F00FF
:103EA00028807878AA1CFFF79EFA387D05F1090270
:103EB00007F11501FFF797FA387B01F048F82874ED
:103EC000787B01F044F86874F87EA874787AE87416
:103ED000387F2875B87B6875388AE882DAF81C0064
:103EE000A861B87A524697F808A0C0F34111012999
:103EF00004D0108C504503D2824609E0FFDF10E069
:103F0000022903D0288820F0600009E0504504D140
:103F1000288820F06000403002E0288840F06000EF
:103F20002880A4F824A0524607F11D01A86996E054
:103F300011264FF02008002C87D0A380686804F178
:103F40000A02007920726868007B607269688B1DC4
:103F500048791946FFF747FAF8E60A264FF0210894
:103F6000002CE9D08888A080686880792072686811
:103F7000C07960729AF8301021F004019FE065E08A
:103F80004CE06FE00B264FF02208002CD4D0C888FC
:103F9000A0806868007920726868007A00F0D7FF16
:103FA00060726868407A00F0D2FFA072CEE61C26EC
:103FB0004FF02608002CBFD0A3806868407960725B
:103FC0006868007AA0720AF1040090E80E00DAF83E
:103FD0001000C4E90530C4E90312686800793C2880
:103FE00003D0432803D0FFDFB0E62772AEE684F8A3
:103FF00008C0ABE610264FF02408002C9CD088881F
:10400000A0806868807920816868807A60816868AB
:104010000089A08168688089E08197E610264FF0CA
:104020002308002C88D08888A0806868C0882081F8
:1040300068680089608168684089A08168688089B3
:10404000E0819AF8301021F0020138E030264FF07C
:104050002508002C85D0A38069682822496821F0B2
:104060008DFA73E614264FF01B08002C8ED0A38027
:10407000686800790128BAD02772DAE90710C4E924
:10408000031063E64A46214660E0287A012803D0FF
:10409000022817D0FFDF59E610264FF01F08002C2A
:1040A00089D06888A080A8892081E8896081288AD1
:1040B000A081688AE0819AF8301021F001018AF825
:1040C000301043E64FF012081026688800F01DFFFC
:1040D0003CE6287AC8B3012838D0022836D0032815
:1040E00001D0FFDF32E609264FF01108002C85D001
:1040F0006F883846FFF7A7F990F822A0A780687A62
:104100002072042138460EF087FC052138460EF057
:1041100083FC002138460EF07FFC012138460EF06A
:104120007BFC032138460EF077FC022138460EF066
:1041300073FC062138460EF06FFC072138460EF05E
:104140006BFC504600F0A7FE00E6FFE72846BDE8FE
:10415000F04701F065BC70B5012803D0052800D0F8
:10416000FFDF70BD8DB22846FFF76DF9040000D166
:10417000FFDF20782128F4D005F0BEF980B1017866
:1041800021F00F01891C21F0F00110310170022192
:10419000017245800020A075BDE8704005F0AFB900
:1041A00021462846BDE870401322FFF74FB92DE99C
:1041B000F04116460C00804600D1FFDF307820F039
:1041C0000F00801C20F0F0001030307020780128A3
:1041D00004D0022818D0FFDFBDE8F0814046FFF789
:1041E00032F9050000D1FFDF0320A87505F087F93B
:1041F00094E80F00083686E80F00FE4810F8301FDC
:1042000041F001010170E7E74046FFF71CF90500A6
:1042100000D1FFDFA1884FF6FF700027814202D155
:10422000E288824203D0814201D1E08840B105F0AA
:1042300066F994E80F00083686E80F00AF75CBE703
:10424000A87D0128C8D178230022414612F04AF8FF
:104250000220A875C0E738B505460C460846FDF7AC
:1042600032F818BB203D062D4AD2DFE805F0031BCB
:10427000373C42300021052012F0B4F808B111207B
:1042800038BDA01C0DF023F904F04CFF050038D117
:10429000002208231146052012F024F8052830D00A
:1042A000FFDF2EE06068FDF752F808B1102038BD3E
:1042B000618820886A460DF0C5FB04F033FF0500D5
:1042C0001FD16068E8B1BDF80010018019E0A07846
:1042D00000F0010120880DF0E6FB0EE0206801F0FF
:1042E0004BFE05460DE0207800F001000CF0EDF9E2
:1042F00003E0618820880DF020FB04F013FFF0E755
:104300000725284638BD70B505460C460846FDF71A
:1043100000F808B1102070BD202D07D0212D0DD040
:10432000222D0BD0252D09D0072070BD2088A11C7F
:104330000CF0A0FABDE8704004F0F4BE062070BD99
:10434000AC482530704708B53421AA4821F0B7F9A8
:104350000120FEF76BFE1120FEF780FEA54968469E
